******************************************************************************
             TMS320C2000 Linker PC v22.6.2                     
******************************************************************************
>> Linked Tue Jun 17 17:35:21 2025

OUTPUT FILE NAME:   <hrpwm_ex2_slider.out>
ENTRY POINT SYMBOL: "code_start"  address: 00000000


MEMORY CONFIGURATION

         name            origin    length      used     unused   attr    fill
----------------------  --------  ---------  --------  --------  ----  --------
PAGE 0:
  BEGIN                 00000000   00000002  00000002  00000000  RWIX
  RAMM0                 000000f6   0000030a  00000030  000002da  RWIX
  RAMLS0                00008000   00000800  00000800  00000000  RWIX
  RAMLS1                00008800   00000800  000007ff  00000001  RWIX
  RAMLS2                00009000   00000800  000000e2  0000071e  RWIX
  RAMLS3                00009800   00000800  00000000  00000800  RWIX
  RAMLS4                0000a000   00000800  00000000  00000800  RWIX
  FLASH_BANK0_SEC0      00080000   00001000  00000000  00001000  RWIX
  FLASH_BANK0_SEC1      00081000   00001000  00000000  00001000  RWIX
  FLASH_BANK0_SEC2      00082000   00001000  00000000  00001000  RWIX
  FLASH_BANK0_SEC3      00083000   00001000  00000000  00001000  RWIX
  FLASH_BANK0_SEC4      00084000   00001000  00000000  00001000  RWIX
  FLASH_BANK0_SEC5      00085000   00001000  00000000  00001000  RWIX
  FLASH_BANK0_SEC6      00086000   00001000  00000000  00001000  RWIX
  FLASH_BANK0_SEC7      00087000   00001000  00000000  00001000  RWIX
  FLASH_BANK0_SEC8      00088000   00001000  00000000  00001000  RWIX
  FLASH_BANK0_SEC9      00089000   00001000  00000000  00001000  RWIX
  FLASH_BANK0_SEC10     0008a000   00001000  00000000  00001000  RWIX
  FLASH_BANK0_SEC11     0008b000   00001000  00000000  00001000  RWIX
  FLASH_BANK0_SEC12     0008c000   00001000  00000000  00001000  RWIX
  FLASH_BANK0_SEC13     0008d000   00001000  00000000  00001000  RWIX
  FLASH_BANK0_SEC14     0008e000   00001000  00000000  00001000  RWIX
  FLASH_BANK0_SEC15     0008f000   00001000  00000000  00001000  RWIX
  FLASH_BANK1_SEC0      00090000   00001000  00000000  00001000  RWIX
  FLASH_BANK1_SEC1      00091000   00001000  00000000  00001000  RWIX
  FLASH_BANK1_SEC2      00092000   00001000  00000000  00001000  RWIX
  FLASH_BANK1_SEC3      00093000   00001000  00000000  00001000  RWIX
  FLASH_BANK1_SEC4      00094000   00001000  00000000  00001000  RWIX
  FLASH_BANK1_SEC5      00095000   00001000  00000000  00001000  RWIX
  FLASH_BANK1_SEC6      00096000   00001000  00000000  00001000  RWIX
  FLASH_BANK1_SEC7      00097000   00001000  00000000  00001000  RWIX
  FLASH_BANK1_SEC8      00098000   00001000  00000000  00001000  RWIX
  FLASH_BANK1_SEC9      00099000   00001000  00000000  00001000  RWIX
  FLASH_BANK1_SEC10     0009a000   00001000  00000000  00001000  RWIX
  FLASH_BANK1_SEC11     0009b000   00001000  00000000  00001000  RWIX
  FLASH_BANK1_SEC12     0009c000   00001000  00000000  00001000  RWIX
  FLASH_BANK1_SEC13     0009d000   00001000  00000000  00001000  RWIX
  FLASH_BANK1_SEC14     0009e000   00001000  00000000  00001000  RWIX
  FLASH_BANK1_SEC15     0009f000   00001000  00000000  00001000  RWIX
  RESET                 003fffc0   00000002  00000000  00000002  RWIX

PAGE 1:
  BOOT_RSVD             00000002   000000f1  00000000  000000f1  RWIX
  RAMM1                 00000400   000003f8  000003f8  00000000  RWIX
  RAMLS5                0000a800   00000800  00000362  0000049e  RWIX
  RAMLS6                0000b000   00000800  00000000  00000800  RWIX
  RAMLS7                0000b800   00000800  00000000  00000800  RWIX
  RAMGS0                0000c000   00002000  00000000  00002000  RWIX
  RAMGS1                0000e000   00002000  00000000  00002000  RWIX
  RAMGS2                00010000   00002000  00000000  00002000  RWIX
  RAMGS3                00012000   00001ff8  00000000  00001ff8  RWIX


SECTION ALLOCATION MAP

 output                                  attributes/
section   page    origin      length       input sections
--------  ----  ----------  ----------   ----------------
codestart 
*          0    00000000    00000002     
                  00000000    00000002     f28004x_codestartbranch.obj (codestart)

.TI.ramfunc 
*          0    000000f6    00000004     
                  000000f6    00000004     driverlib_eabi.lib : sysctl.obj (.TI.ramfunc)

.cinit     0    000000fa    0000002c     
                  000000fa    0000001a     (.cinit..data.load) [load image, compression = lzss]
                  00000114    00000006     (__TI_handler_table)
                  0000011a    00000004     (.cinit..bss.load) [load image, compression = zero_init]
                  0000011e    00000008     (__TI_cinit_table)

.reset     0    003fffc0    00000000     DSECT

.stack     1    00000400    000003f8     UNINITIALIZED
                  00000400    000003f8     --HOLE--

.bss       1    0000ab53    00000010     UNINITIALIZED
                  0000ab53    00000009     SFO_v8_fpu_lib_build_c28_driverlib_eabi.lib : SFO_v8_fpu_lib_build_c28_driverlib.obj (.bss:MEP_SF)
                  0000ab5c    00000005                                                 : SFO_v8_fpu_lib_build_c28_driverlib.obj (.bss)
                  0000ab61    00000001     c2000ware_libraries.obj (.bss)
                  0000ab62    00000001     hrpwm_ex2_slider.obj (.bss)

.init_array 
*          0    000000f6    00000000     UNINITIALIZED

.const     1    0000a800    00000337     
                  0000a800    000000cd     board.obj (.const:.string)
                  0000a8cd    00000001     --HOLE-- [fill = 0]
                  0000a8ce    0000009a     driverlib_eabi.lib : sysctl.obj (.const:.string)
                  0000a968    00000098                        : epwm.obj (.const:.string)
                  0000aa00    00000098                        : gpio.obj (.const:.string)
                  0000aa98    00000059     device.obj (.const:.string)
                  0000aaf1    00000001     --HOLE-- [fill = 0]
                  0000aaf2    00000045     hrpwm_ex2_slider.obj (.const:.string)

.data      1    0000ab38    0000001b     UNINITIALIZED
                  0000ab38    00000010     c2000ware_libraries.obj (.data:ePWM)
                  0000ab48    00000006     rts2800_fpu32_eabi.lib : exit.c.obj (.data)
                  0000ab4e    00000002                            : _lock.c.obj (.data:_lock)
                  0000ab50    00000002                            : _lock.c.obj (.data:_unlock)
                  0000ab52    00000001     SFO_v8_fpu_lib_build_c28_driverlib_eabi.lib : SFO_v8_fpu_lib_build_c28_driverlib.obj (.data)

.text.1    0    00008000    00000800     
                  00008000    000001f1     SFO_v8_fpu_lib_build_c28_driverlib_eabi.lib : SFO_v8_fpu_lib_build_c28_driverlib.obj (.text:SFO)
                  000081f1    000000f6     board.obj (.text:EPWM_init)
                  000082e7    000000dc     device.obj (.text:Device_enableAllPeripherals)
                  000083c3    000000c8     driverlib_eabi.lib : sysctl.obj (.text:SysCtl_setClock)
                  0000848b    000000bd                        : sysctl.obj (.text:SysCtl_isPLLValid)
                  00008548    00000073                        : sysctl.obj (.text:DCC_setCounterSeeds)
                  000085bb    0000005e                        : sysctl.obj (.text:SysCtl_getClock)
                  00008619    00000052                        : gpio.obj (.text:GPIO_setPadConfig)
                  0000866b    00000051     device.obj (.text:Device_init)
                  000086bc    0000004d     driverlib_eabi.lib : sysctl.obj (.text:SysCtl_selectOscSource)
                  00008709    00000045                        : sysctl.obj (.text:SysCtl_pollX1Counter)
                  0000874e    00000045     hrpwm_ex2_slider.obj (.text:main)
                  00008793    00000040     board.obj (.text:EPWM_setActionQualifierAction)
                  000087d3    0000002c     board.obj (.text:EPWM_setDeadBandDelayMode)
                  000087ff    00000001     rts2800_fpu32_eabi.lib : startup.c.obj (.text)

.text.2    0    00008800    000007ff     
                  00008800    00000040     driverlib_eabi.lib : sysctl.obj (.text:SysCtl_selectXTAL)
                  00008840    0000003e     board.obj (.text:EPWM_setCounterCompareShadowLoadMode)
                  0000887e    0000003d     driverlib_eabi.lib : interrupt.obj (.text:Interrupt_initModule)
                  000088bb    0000003a                        : gpio.obj (.text:GPIO_setAnalogMode)
                  000088f5    00000037                        : gpio.obj (.text:GPIO_setPinConfig)
                  0000892c    00000037                        : gpio.obj (.text:GPIO_setQualificationMode)
                  00008963    00000031                        : gpio.obj (.text:GPIO_setDirectionMode)
                  00008994    0000002e     rts2800_fpu32_eabi.lib : copy_decompress_lzss.c.obj (.text:decompress:lzss)
                  000089c2    0000002b     board.obj (.text:EPWM_isBaseValid)
                  000089ed    0000002b     driverlib_eabi.lib : epwm.obj (.text:EPWM_isBaseValid)
                  00008a18    0000002b     board.obj (.text:HRPWM_isBaseValid)
                  00008a43    0000002b     hrpwm_ex2_slider.obj (.text:HRPWM_isBaseValid)
                  00008a6e    0000002b     rts2800_fpu32_eabi.lib : autoinit.c.obj (.text:__TI_auto_init_nobinit_nopinit)
                  00008a99    00000029                            : exit.c.obj (.text)
                  00008ac2    00000027     board.obj (.text:EPWM_setSyncOutPulseMode)
                  00008ae9    00000027     board.obj (.text:HRPWM_setCounterCompareShadowLoadEvent)
                  00008b10    00000027     board.obj (.text:SysCtl_setSyncInputConfig)
                  00008b37    00000025     driverlib_eabi.lib : sysctl.obj (.text:SysCtl_selectXTALSingleEnded)
                  00008b5c    00000024                        : sysctl.obj (.text:DCC_enableSingleShotMode)
                  00008b80    00000022     board.obj (.text:EPWM_setCounterCompareValue)
                  00008ba2    00000022     board.obj (.text:HRPWM_setMEPEdgeSelect)
                  00008bc4    00000020     board.obj (.text:XBAR_setInputPin)
                  00008be4    0000001f     board.obj (.text:EPWM_setFallingEdgeDelayCountShadowLoadMode)
                  00008c03    0000001f     board.obj (.text:EPWM_setRisingEdgeDelayCountShadowLoadMode)
                  00008c22    0000001f     board.obj (.text:HRPWM_setFallingEdgeDelayLoadMode)
                  00008c41    0000001f     board.obj (.text:HRPWM_setPhaseShift)
                  00008c60    0000001f     board.obj (.text:HRPWM_setRisingEdgeDelayLoadMode)
                  00008c7f    0000001e     driverlib_eabi.lib : sysctl.obj (.text:DCC_setCounter1ClkSource)
                  00008c9d    0000001e     hrpwm_ex2_slider.obj (.text:HRPWM_setHiResFallingEdgeDelayOnly)
                  00008cbb    0000001e     driverlib_eabi.lib : interrupt.obj (.text:Interrupt_initVectorTable)
                  00008cd9    0000001e     board.obj (.text:PinMux_init)
                  00008cf7    0000001e     board.obj (.text:SYNC_init)
                  00008d15    0000001d     board.obj (.text:EPWM_setDeadBandCounterClock)
                  00008d32    0000001d     board.obj (.text:EPWM_setFallingEdgeDelayCount)
                  00008d4f    0000001d     board.obj (.text:EPWM_setRisingEdgeDelayCount)
                  00008d6c    0000001d     rts2800_fpu32_eabi.lib : memcpy.c.obj (.text)
                  00008d89    0000001c     driverlib_eabi.lib : sysctl.obj (.text:DCC_setCounter0ClkSource)
                  00008da5    0000001c     board.obj (.text:EPWM_setClockPrescaler)
                  00008dc1    0000001c     board.obj (.text:HRPWM_setDeadbandMEPEdgeSelect)
                  00008ddd    0000001a     driverlib_eabi.lib : sysctl.obj (.text:SysCtl_getLowSpeedClock)
                  00008df7    00000018     hrpwm_ex2_slider.obj (.text:SysCtl_disablePeripheral)
                  00008e0f    00000017     device.obj (.text:SysCtl_enablePeripheral)
                  00008e26    00000017     driverlib_eabi.lib : sysctl.obj (.text:SysCtl_enablePeripheral)
                  00008e3d    00000017     hrpwm_ex2_slider.obj (.text:SysCtl_enablePeripheral)
                  00008e54    00000017     rts2800_fpu32_eabi.lib : boot28.asm.obj (.text)
                  00008e6b    00000016     driverlib_eabi.lib : sysctl.obj (.text:DCC_disableDoneSignal)
                  00008e81    00000016                        : sysctl.obj (.text:DCC_enableDoneSignal)
                  00008e97    00000016                        : epwm.obj (.text:EPWM_setEmulationMode)
                  00008ead    00000016                        : interrupt.obj (.text:Interrupt_defaultHandler)
                  00008ec3    00000015                        : sysctl.obj (.text:DCC_clearDoneFlag)
                  00008ed8    00000015                        : sysctl.obj (.text:DCC_clearErrorFlag)
                  00008eed    00000015                        : sysctl.obj (.text:DCC_disableErrorSignal)
                  00008f02    00000015                        : sysctl.obj (.text:DCC_enableErrorSignal)
                  00008f17    00000015     device.obj (.text:GPIO_unlockPortConfig)
                  00008f2c    00000015     board.obj (.text:HRPWM_disablePhaseShiftLoad)
                  00008f41    00000015     board.obj (.text:HRPWM_enableAutoConversion)
                  00008f56    00000014     driverlib_eabi.lib : sysctl.obj (.text:DCC_disableModule)
                  00008f6a    00000014                        : sysctl.obj (.text:DCC_enableModule)
                  00008f7e    00000014     board.obj (.text:EPWM_setTimeBaseCounterMode)
                  00008f92    00000014     board.obj (.text:EPWM_setTimeBasePeriod)
                  00008fa6    00000014     driverlib_eabi.lib : gpio.obj (.text:GPIO_isPinValid)
                  00008fba    00000014     device.obj (.text:SysCtl_deviceCal)
                  00008fce    00000012     board.obj (.text:EPWM_setTimeBaseCounter)
                  00008fe0    00000012     board.obj (.text:SysCtl_setSyncOutputConfig)
                  00008ff2    0000000d     driverlib_eabi.lib : interrupt.obj (.text:Interrupt_disableGlobal)

.text.3    0    00009000    000000e2     
                  00009000    00000011     board.obj (.text:EPWM_disablePhaseShiftLoad)
                  00009011    00000010     driverlib_eabi.lib : sysctl.obj (.text:DCC_isBaseValid)
                  00009021    00000010     device.obj (.text:Device_initGPIO)
                  00009031    0000000f     device.obj (.text:ASysCtl_disableDCDC)
                  00009040    0000000d     device.obj (.text:SysCtl_setLowSpeedClock)
                  0000904d    0000000d     rts2800_fpu32_eabi.lib : copy_zero_init.c.obj (.text:decompress:ZI:__TI_zero_init_nomemset)
                  0000905a    0000000c     board.obj (.text:SysCtl_enableExtADCSOCSource)
                  00009066    0000000c     rts2800_fpu32_eabi.lib : args_main.c.obj (.text)
                  00009072    0000000b     board.obj (.text:Board_init)
                  0000907d    0000000b     device.obj (.text:SysCtl_disableWatchdog)
                  00009088    0000000b     driverlib_eabi.lib : sysctl.obj (.text:SysCtl_isMCDClockFailureDetected)
                  00009093    0000000a                        : interrupt.obj (.text:Interrupt_illegalOperationHandler)
                  0000909d    0000000a                        : interrupt.obj (.text:Interrupt_nmiHandler)
                  000090a7    00000009     rts2800_fpu32_eabi.lib : _lock.c.obj (.text)
                  000090b0    00000008                            : copy_decompress_none.c.obj (.text:decompress:none)
                  000090b8    00000008     f28004x_codestartbranch.obj (.text)
                  000090c0    00000007     driverlib_eabi.lib : sysctl.obj (.text:SysCtl_resetMCD)
                  000090c7    00000007     device.obj (.text:__error__)
                  000090ce    00000005     board.obj (.text:INPUTXBAR_init)
                  000090d3    00000005     board.obj (.text:myINPUTXBARINPUT0_init)
                  000090d8    00000005     board.obj (.text:myINPUTXBARINPUT1_init)
                  000090dd    00000003     hrpwm_ex2_slider.obj (.text:error)
                  000090e0    00000002     rts2800_fpu32_eabi.lib : pre_init.c.obj (.text)

MODULE SUMMARY

       Module                                   code   ro data   rw data
       ------                                   ----   -------   -------
    .\
       hrpwm_ex2_slider.obj                     192    69        1      
    +--+----------------------------------------+------+---------+---------+
       Total:                                   192    69        1      
                                                                        
    .\device\
       device.obj                               427    89        0      
       f28004x_codestartbranch.obj              10     0         0      
    +--+----------------------------------------+------+---------+---------+
       Total:                                   437    89        0      
                                                                        
    .\syscfg\
       board.obj                                1250   205       0      
       c2000ware_libraries.obj                  0      0         17     
    +--+----------------------------------------+------+---------+---------+
       Total:                                   1250   205       17     
                                                                        
    C:\ti\c2000\C2000Ware_5_04_00_00\driverlib\f28004x\driverlib\ccs\Debug\driverlib_eabi.lib
       sysctl.obj                               1194   154       0      
       gpio.obj                                 319    152       0      
       epwm.obj                                 65     152       0      
       interrupt.obj                            146    0         0      
    +--+----------------------------------------+------+---------+---------+
       Total:                                   1724   458       0      
                                                                        
    C:\ti\c2000\C2000Ware_5_04_00_00\libraries\calibration\hrpwm\f28004x\lib\SFO_v8_fpu_lib_build_c28_driverlib_eabi.lib
       SFO_v8_fpu_lib_build_c28_driverlib.obj   497    0         15     
    +--+----------------------------------------+------+---------+---------+
       Total:                                   497    0         15     
                                                                        
    C:\ti\ccs2020\ccs\tools\compiler\ti-cgt-c2000_22.6.2.LTS\lib\rts2800_fpu32_eabi.lib
       exit.c.obj                               41     0         6      
       copy_decompress_lzss.c.obj               46     0         0      
       autoinit.c.obj                           43     0         0      
       memcpy.c.obj                             29     0         0      
       boot28.asm.obj                           23     0         0      
       _lock.c.obj                              9      0         4      
       copy_zero_init.c.obj                     13     0         0      
       args_main.c.obj                          12     0         0      
       copy_decompress_none.c.obj               8      0         0      
       pre_init.c.obj                           2      0         0      
       startup.c.obj                            1      0         0      
    +--+----------------------------------------+------+---------+---------+
       Total:                                   227    0         10     
                                                                        
       Stack:                                   0      0         1016   
       Linker Generated:                        0      44        0      
    +--+----------------------------------------+------+---------+---------+
       Grand Total:                             4327   865       1059   


LINKER GENERATED COPY TABLES

__TI_cinit_table @ 0000011e records: 2, size/record: 4, table size: 8
	.data: load addr=000000fa, load size=0000001a bytes, run addr=0000ab38, run size=0000001b bytes, compression=lzss
	.bss: load addr=0000011a, load size=00000004 bytes, run addr=0000ab53, run size=00000010 bytes, compression=zero_init


LINKER GENERATED HANDLER TABLE

__TI_handler_table @ 00000114 records: 3, size/record: 2, table size: 6
	index: 0, handler: __TI_zero_init
	index: 1, handler: __TI_decompress_lzss
	index: 2, handler: __TI_decompress_none


GLOBAL DATA SYMBOLS: SORTED BY DATA PAGE

address     data page           name
--------    ----------------    ----
00000400      10 (00000400)     __stack

0000ab38     2ac (0000ab00)     ePWM

0000ab48     2ad (0000ab40)     __TI_enable_exit_profile_output
0000ab4a     2ad (0000ab40)     __TI_cleanup_ptr
0000ab4c     2ad (0000ab40)     __TI_dtors_ptr
0000ab4e     2ad (0000ab40)     _lock
0000ab50     2ad (0000ab40)     _unlock
0000ab53     2ad (0000ab40)     MEP_SF
0000ab5c     2ad (0000ab40)     SFO_CAL
0000ab61     2ad (0000ab40)     MEP_ScaleFactor
0000ab62     2ad (0000ab40)     status


GLOBAL SYMBOLS: SORTED ALPHABETICALLY BY Name 

page  address   name                             
----  -------   ----                             
0     00009072  Board_init                       
0     00008a99  C$$EXIT                          
0     000082e7  Device_enableAllPeripherals      
0     0000866b  Device_init                      
0     00009021  Device_initGPIO                  
0     000081f1  EPWM_init                        
0     00008e97  EPWM_setEmulationMode            
0     000088bb  GPIO_setAnalogMode               
0     00008963  GPIO_setDirectionMode            
0     00008619  GPIO_setPadConfig                
0     000088f5  GPIO_setPinConfig                
0     0000892c  GPIO_setQualificationMode        
0     000090ce  INPUTXBAR_init                   
0     00008ead  Interrupt_defaultHandler         
0     00009093  Interrupt_illegalOperationHandler
0     0000887e  Interrupt_initModule             
0     00008cbb  Interrupt_initVectorTable        
0     0000909d  Interrupt_nmiHandler             
1     0000ab53  MEP_SF                           
1     0000ab61  MEP_ScaleFactor                  
0     00008cd9  PinMux_init                      
0     00008000  SFO                              
1     0000ab5c  SFO_CAL                          
0     00008cf7  SYNC_init                        
0     000000f6  SysCtl_delay                     
0     000085bb  SysCtl_getClock                  
0     00008ddd  SysCtl_getLowSpeedClock          
0     0000848b  SysCtl_isPLLValid                
0     000086bc  SysCtl_selectOscSource           
0     00008800  SysCtl_selectXTAL                
0     00008b37  SysCtl_selectXTALSingleEnded     
0     000083c3  SysCtl_setClock                  
0     0000011e  __TI_CINIT_Base                  
0     00000126  __TI_CINIT_Limit                 
0     00000126  __TI_CINIT_Warm                  
0     00000114  __TI_Handler_Table_Base          
0     0000011a  __TI_Handler_Table_Limit         
1     000007f8  __TI_STACK_END                   
abs   000003f8  __TI_STACK_SIZE                  
0     00008a6e  __TI_auto_init_nobinit_nopinit   
1     0000ab4a  __TI_cleanup_ptr                 
0     00008994  __TI_decompress_lzss             
0     000090b0  __TI_decompress_none             
1     0000ab4c  __TI_dtors_ptr                   
1     0000ab48  __TI_enable_exit_profile_output  
abs   ffffffff  __TI_pprof_out_hndl              
abs   ffffffff  __TI_prof_data_size              
abs   ffffffff  __TI_prof_data_start             
0     0000904d  __TI_zero_init_nomemset          
n/a   UNDEFED   __c_args__                       
0     000090c7  __error__                        
1     00000400  __stack                          
0     00009066  _args_main                       
0     00008e54  _c_int00                         
1     0000ab4e  _lock                            
0     000090af  _nop                             
0     000090ab  _register_lock                   
0     000090a7  _register_unlock                 
0     000087ff  _system_post_cinit               
0     000090e0  _system_pre_init                 
1     0000ab50  _unlock                          
0     00008a99  abort                            
0     00000000  code_start                       
1     0000ab38  ePWM                             
0     000090dd  error                            
0     00008a9b  exit                             
0     0000874e  main                             
0     00008d6c  memcpy                           
0     000090d3  myINPUTXBARINPUT0_init           
0     000090d8  myINPUTXBARINPUT1_init           
1     0000ab62  status                           


GLOBAL SYMBOLS: SORTED BY Symbol Address 

page  address   name                             
----  -------   ----                             
0     00000000  code_start                       
0     000000f6  SysCtl_delay                     
0     00000114  __TI_Handler_Table_Base          
0     0000011a  __TI_Handler_Table_Limit         
0     0000011e  __TI_CINIT_Base                  
0     00000126  __TI_CINIT_Limit                 
0     00000126  __TI_CINIT_Warm                  
0     00008000  SFO                              
0     000081f1  EPWM_init                        
0     000082e7  Device_enableAllPeripherals      
0     000083c3  SysCtl_setClock                  
0     0000848b  SysCtl_isPLLValid                
0     000085bb  SysCtl_getClock                  
0     00008619  GPIO_setPadConfig                
0     0000866b  Device_init                      
0     000086bc  SysCtl_selectOscSource           
0     0000874e  main                             
0     000087ff  _system_post_cinit               
0     00008800  SysCtl_selectXTAL                
0     0000887e  Interrupt_initModule             
0     000088bb  GPIO_setAnalogMode               
0     000088f5  GPIO_setPinConfig                
0     0000892c  GPIO_setQualificationMode        
0     00008963  GPIO_setDirectionMode            
0     00008994  __TI_decompress_lzss             
0     00008a6e  __TI_auto_init_nobinit_nopinit   
0     00008a99  C$$EXIT                          
0     00008a99  abort                            
0     00008a9b  exit                             
0     00008b37  SysCtl_selectXTALSingleEnded     
0     00008cbb  Interrupt_initVectorTable        
0     00008cd9  PinMux_init                      
0     00008cf7  SYNC_init                        
0     00008d6c  memcpy                           
0     00008ddd  SysCtl_getLowSpeedClock          
0     00008e54  _c_int00                         
0     00008e97  EPWM_setEmulationMode            
0     00008ead  Interrupt_defaultHandler         
0     00009021  Device_initGPIO                  
0     0000904d  __TI_zero_init_nomemset          
0     00009066  _args_main                       
0     00009072  Board_init                       
0     00009093  Interrupt_illegalOperationHandler
0     0000909d  Interrupt_nmiHandler             
0     000090a7  _register_unlock                 
0     000090ab  _register_lock                   
0     000090af  _nop                             
0     000090b0  __TI_decompress_none             
0     000090c7  __error__                        
0     000090ce  INPUTXBAR_init                   
0     000090d3  myINPUTXBARINPUT0_init           
0     000090d8  myINPUTXBARINPUT1_init           
0     000090dd  error                            
0     000090e0  _system_pre_init                 
1     00000400  __stack                          
1     000007f8  __TI_STACK_END                   
1     0000ab38  ePWM                             
1     0000ab48  __TI_enable_exit_profile_output  
1     0000ab4a  __TI_cleanup_ptr                 
1     0000ab4c  __TI_dtors_ptr                   
1     0000ab4e  _lock                            
1     0000ab50  _unlock                          
1     0000ab53  MEP_SF                           
1     0000ab5c  SFO_CAL                          
1     0000ab61  MEP_ScaleFactor                  
1     0000ab62  status                           
abs   000003f8  __TI_STACK_SIZE                  
abs   ffffffff  __TI_pprof_out_hndl              
abs   ffffffff  __TI_prof_data_size              
abs   ffffffff  __TI_prof_data_start             
n/a   UNDEFED   __c_args__                       

[71 symbols]
